:020000040000FA
:10000000831285018601870183160B3085008601E6
:10001000870110309F008312031703309E009F0159
:100020000313C1309F00A001A101A201A3010A3066
:10003000A5008613200831208700051683200512AD
:100040002108312087000515832005112208312061
:10005000870086178320A503031D19283F205E20F3
:1000600017280F3982073F340A345D345E346A340E
:10007000763477341A347F347E34403435349F14E8
:100080009F18402883161E088312A3001E08A40090
:100090000800FF30A000A1006430A00AA302030101
:1000A000031C013EA40203184C2864302307F63ECB
:1000B000A10A031857280A3EA20008006030A302D4
:1000C0000130031C013EA40203186A280A30A00074
:1000D000A1000800230803178D0083168C130C144D
:1000E00083120C080313A000A100A300A00E0F3080
:1000F000A005A1050B30A2002530230203188516A8
:10010000031C851208000630A600FA30FF3E031DCE
:080110008628A60B85280800D3
:02400E00C430BC
:10420000F034F034F034F134F134F134F134F13489
:10421000F234F234F234F234F234F334F334F3346B
:10422000F334F334F434F434F434F434F434F5344F
:10423000F534F534F534F534F534F634F634F63433
:10424000F634F634F734F734F734F734F734F83417
:10425000F834F834F834F834F934F934F934F934FA
:10426000F934103410341034103410341134113443
:104270001134113411341134123412341234123412
:1042800012341334133413341334133414341434F5
:1042900014341434143415341534153415341534D9
:1042A00016341634163416341634163417341734BC
:1042B00017341734173418341834183418341834A1
:1042C0001934193419341934193420342034203471
:1042D0002034203421342134213421342134223437
:1042E000223422342234223422342334233423341B
:1042F00023342334243424342434243424342534FF
:1043000025342534253425342634263426342634E1
:1043100026342734273427342734273427342834C5
:1043200028342834283428342934293429342934A9
:104330002934303430343034303430343134313462
:104340003134313431343234323432343234323440
:104350003334333433343334333433343434343423
:104360003434343434343534353435343534353408
:1043700036343634363436343634373437343734EA
:1043800037343734383438343834383438343834CF
:1043900039343934393439343934403440344034A0
:1043A0004034403441344134413441344134423466
:1043B0004234423442344234433443344334433449
:1043C000433444344434443444344434443445342D
:1043D0004534453445344534463446344634463411
:1043E00046344734473447344734473448344834F4
:1043F00048344834483449344934493449344934D8
:00000001FF
